:020000040000FA
:100000000C947F000C94A7000C94A7000C94A700FC
:100010000C94A7000C94A7000C94A7000C94A700C4
:100020000C94A7000C94A7000C94A7000C94A700B4
:100030000C94A7000C94A7000C94A7000C94A700A4
:100040000C94F8040C94A7000C94C6040C94A0041F
:100050000C94A7000C94A7000C94A7000C94A70084
:100060000C94A7000C94A70050000000000024008E
:1000700027002A00486F6D65536572766572494F97
:100080004578742076007D002C2248223A007B229D
:1000900054223A004552523A20444854206661693D
:1000A0006C656420746F207265616400000000005C
:1000B000250028002B0000000008000201000003BA
:1000C0000407000000000000000000000000230002
:1000D00026002900040404040404040402020202A9
:1000E00002020303030303030102040810204080FB
:1000F0000102040810200102040810204205112406
:100100001FBECFEFD8E0DEBFCDBF11E0A0E0B1E071
:10011000E4EDF4E102C005900D92A832B107D9F7E1
:1001200021E0A8E2B1E001C01D92A73FB207E1F7CC
:1001300010E0CFE7D0E004C02197FE010E94620AE0
:10014000CE37D107C9F70E948F050C94680A0C942A
:100150000000CF92DF92EF92FF92CF93DF93B091A6
:10016000EB01A0E08111AB2F8091EC0190E0880FB2
:10017000991FAC0146535F4FC090F101D090F2013E
:10018000E090F301F090F40130E020E0FA01C59135
:10019000D491E881B90190E080E0EB23EA130AC032
:1001A0002F5F3F4F6C157D058E059F0578F36FEF30
:1001B0007FEFCB01DF91CF91FF90EF90DF90CF9059
:1001C0000895AF92BF92CF92DF92EF92FF920F937A
:1001D0001F93CF93DF936C017B018B01040F151FDD
:1001E000EB015E01AE18BF08C017D10759F0699145
:1001F000D601ED91FC910190F081E02DC6010995A9
:10020000892B79F7C501DF91CF911F910F91FF9055
:10021000EF90DF90CF90BF90AF900895FC01538D89
:10022000448D252F30E0842F90E0821B930B5417D0
:1002300010F0CF96089501970895FC01918D828D5D
:10024000981761F0A28DAE0FBF2FB11D5D968C91F6
:10025000928D9F5F9F73928F90E008958FEF9FEF35
:100260000895FC01918D828D981731F0828DE80FF1
:10027000F11D858D90E008958FEF9FEF0895FC01AB
:10028000918D228D892F90E0805C9F4F821B910978
:100290008F739927089587E491E00E943F0121E040
:1002A000892B09F420E0822F089580E090E0892BCB
:1002B00029F00E944B0181110C9400000895FC016B
:1002C000A48DA80FB92FB11DA35ABF4F2C91848DB7
:1002D00090E001968F739927848FA689B7892C9314
:1002E000A089B1898C91837080648C93938D848D67
:1002F000981306C00288F389E02D80818F7D80836A
:100300000895EF92FF920F931F93CF93DF93EC0129
:1003100081E0888F9B8D8C8D98131AC0E889F989AC
:10032000808185FF15C09FB7F894EE89FF896083AF
:10033000E889F98980818370806480839FBF81E030
:1003400090E0DF91CF911F910F91FF90EF90089572
:10035000F62E0B8D10E00F5F1F4F0F731127E02E4D
:100360008C8D8E110CC00FB607FCFACFE889F98985
:10037000808185FFF5CFCE010E945F01F1CFEB8D2B
:10038000EC0FFD2FF11DE35AFF4FF0829FB7F89459
:100390000B8FEA89FB8980818062CFCF0F931F93F7
:1003A000CF93DF938C01D0E0C0E0F801EC0FFD1F8C
:1003B0006491662341F087E491E00E948101892BDA
:1003C00011F02196F2CFCE01DF91CF911F910F91C5
:1003D0000895CF93DF93EC01888D8823B9F0AA8923
:1003E000BB89E889F9898C9185FD03C0808186FDF0
:1003F0000DC00FB607FCF7CF8C9185FFF2CF80813F
:1004000085FFEDCFCE010E945F01E9CFDF91CF9153
:100410000895833081F028F4813099F08230A9F07A
:1004200008958730A9F08830C9F08430B1F4809104
:1004300080008F7D03C0809180008F778093800043
:10044000089584B58F7784BD089584B58F7DFBCFE3
:100450008091B0008F778093B00008958091B000B4
:100460008F7DF9CFCF93DF93282F30E0F901EA5445
:10047000FF4F8491F901E851FF4FD491F901EC52FB
:10048000FF4FC491CC23A1F081110E940902EC2FEF
:10049000F0E0EE0FFF1FE653FF4FA591B491EC91F2
:1004A000ED2381E090E009F480E0DF91CF910895A1
:1004B00080E090E0FACFCF93DF9390E0FC01E85129
:1004C000FF4F24918C529F4FFC0184918823D1F0DF
:1004D00090E0880F991FFC01E659FF4FA591B49158
:1004E000FC01E455FF4FC591D491623071F49FB780
:1004F000F8943C91822F809583238C93E8812E2B56
:1005000028839FBFDF91CF9108958FB7F894EC9126
:100510002E2B2C938FBFF6CF3FB7F89480912D01EF
:1005200090912E01A0912F01B091300126B5A89B8A
:1005300005C02F3F19F00196A11DB11D3FBFBA2F75
:10054000A92F982F8827BC01CD01620F711D811D35
:10055000911D42E0660F771F881F991F4A95D1F7BA
:1005600008958F929F92AF92BF92CF92DF92EF92B7
:10057000FF924B015C010E948C026B017C010E9486
:100580008C026C197D098E099F09683E73408105B4
:100590009105A8F321E0821A9108A108B10888EE1C
:1005A000C80E83E0D81EE11CF11C81149104A10443
:1005B000B10429F7FF90EF90DF90CF90BF90AF90FC
:1005C0009F908F9008952FB7F894609129017091B2
:1005D0002A0180912B0190912C012FBF08958F92B9
:1005E0009F92AF92BF92CF92DF92EF92FF920F93C2
:1005F0001F93CF93DF93CDB7DEB7C054D1400FB672
:10060000F894DEBF0FBECDBF0E94E3020091ED0162
:100610001091EE012091EF013091F0016B017C010E
:10062000C01AD10AE20AF30A97018601003D174079
:1006300021053105B0F48091F501C05CDE4F0FB6A5
:10064000F894DEBF0FBECDBFDF91CF911F910F9108
:10065000FF90EF90DF90CF90BF90AF909F908F90E2
:1006600008956093ED017093EE018093EF019093F4
:10067000F0011092E8011092E7011092E601109249
:10068000E5011092E40162E08091E9010E945B02C1
:1006900061E070E080E090E00E94B10261E0809152
:1006A000E9010E945B022091E90130E0F901EA547E
:1006B000FF4F8491F901E851FF4F0491F901EC5289
:1006C000FF4F1491112391F081110E940902E12F33
:1006D000F0E0EE0FFF1FE455FF4FA591B4918FB7E7
:1006E000F894EC9100950E230C938FBF8091EA0152
:1006F0008551823020F58BE291E10197F1F762E0BC
:100700008091E9010E945B028091F60190E08230C5
:10071000910538F0880F991F880F991F0597019749
:10072000F1F7F89480E00E94A9006F3F7F4F8F4F50
:100730009F4F61F41092F501789480E07ECF64E1E0
:1007400070E080E090E00E94B102D9CF81E00E9489
:10075000A9006F3F7F4F8F4F9F4F61F3CE010196EE
:100760007C015E019FEBA91A9EEFB90A870180E028
:100770000E94A900F801608371838283938381E0E2
:100780000E94A900F8016483758386839783085FBC
:100790001F4FA016B10659F7789430E020E0F7011A
:1007A00080809180A280B380448155816681778169
:1007B000FFEF8F169F06AF06BF0631F04F3F8FEF5A
:1007C00058076807780719F41092F501B6CFF901B8
:1007D00083E0F595E7958A95E1F7EC51FE4F80812E
:1007E000880F84169506A606B70618F180832F5F3A
:1007F0003F4F98E0E90EF11C2832310581F6409117
:10080000E8012091E4018091E501280F3327331F8F
:100810008091E601280F311D8091E701820F932F0F
:10082000911D99274817190679F681E08093F50103
:1008300004CF8160DBCFFC0101900020E9F7319704
:10084000AF01481B590BBC0187E491E00C94E10017
:100850008F929F92AF92BF920F931F93CF93DF938C
:10086000CDB7DEB7A1970FB6F894DEBF0FBECDBFF0
:1008700019A2423008F44AE08E010F5D1F4F842E0A
:10088000912CB12CA12CA50194010E94400AE62FC5
:10089000B901CA01EA30F4F4E05DD801EE938D01AC
:1008A000232B242B252B79F790E080E0109719F06B
:1008B000CD010E941B04A1960FB6F894DEBF0FBEB7
:1008C000CDBFDF91CF911F910F91BF90AF909F90BF
:1008D0008F900895E95CE1CFCF93DF930E941B04D2
:1008E000EC0182E191E00E941B048C0F9D1FDF91BF
:1008F000CF910895CF93C82F88E690E00E94CE0153
:100900006C2F70E090E080E04AE00E94280485E1CE
:1009100091E00E941B04EC2FF0E0E15DFE4F80812E
:10092000882359F087E191E00E946C0465E070E053
:1009300080E090E0CF910C94B10289E191E0F4CF96
:100940001F920F920FB60F9211242F933F934F9344
:100950005F936F937F938F939F93AF93BF93EF9327
:10096000FF9387E491E00E945F01FF91EF91BF91B7
:10097000AF919F918F917F916F915F914F913F9137
:100980002F910F900FBE0F901F9018951F920F92EE
:100990000FB60F9211242F938F939F93EF93FF9392
:1009A000E0915701F09158018081E0915D01F09153
:1009B0005E0182FD1BC09081809160018F5F8F730B
:1009C00020916101821741F0E0916001F0E0E95B64
:1009D000FE4F958F80936001FF91EF919F918F91D2
:1009E0002F910F900FBE0F901F9018958081F4CF1C
:1009F0001F920F920FB60F9211242F933F938F9354
:100A00009F93AF93BF938091290190912A01A09168
:100A10002B01B0912C013091280123E0230F2D37B9
:100A200058F50196A11DB11D20932801809329013D
:100A300090932A01A0932B01B0932C0180912D015A
:100A400090912E01A0912F01B09130010196A11D2E
:100A5000B11D80932D0190932E01A0932F01B0938F
:100A60003001BF91AF919F918F913F912F910F9046
:100A70000FBE0F901F90189526E8230F0296A11D18
:100A8000B11DD2CFE7E4F1E01382128288EE93E049
:100A9000A0E0B0E084839583A683B78384E091E0EF
:100AA0009183808385EC90E09587848784EC90E047
:100AB0009787868780EC90E0918B808B81EC90E02B
:100AC000938B828B82EC90E0958B848B86EC90E00C
:100AD000978B868B118E128E138E148EA4EEB1E03E
:100AE00081E115968C93159786E116968C9316974F
:100AF000E9EFF0E0E4911796EC931797E5EEF0E05C
:100B0000E4911896EC93189740E85EE360E070E09B
:100B10001D964D935D936D937C93509708957894B3
:100B200084B5826084BD84B5816084BD85B58260F2
:100B300085BD85B5816085BD80916E0081608093A3
:100B40006E0010928100809181008260809381000C
:100B5000809181008160809381008091800081601C
:100B6000809380008091B10084608093B100809177
:100B7000B00081608093B00080917A00846080939F
:100B80007A0080917A00826080937A0080917A0066
:100B9000816080937A0080917A00806880937A00E7
:100BA0001092C100E0915701F091580182E08083DA
:100BB000E0915701F09158011082E0915301F091BA
:100BC00054011082E0915501F091560180E180833B
:100BD00010925F01E0915B01F0915C0186E08083FF
:100BE000E0915901F0915A01808180618083E09108
:100BF0005901F0915A01808188608083E091590108
:100C0000F0915A01808180688083E0915901F091D0
:100C10005A0180818F7D808384E790E00E94CE011D
:100C20008BE191E00E946C0462E082E00E945B0232
:100C300062E083E00E945B0262E084E00E945B026B
:100C400082E00E94320221E0892B09F420E0209307
:100C5000310183E00E94320221E0892B09F420E077
:100C60002093320184E00E94320221E0892B09F4B2
:100C700020E02093330162E08091E9010E945B0251
:100C80000E94E302605D7740810991096093ED0164
:100C90007093EE018093EF019093F00187E38093CE
:100CA000F601C0E0D0E030E4A32E31E0B32E41E302
:100CB000C42E41E0D42E54E3E52E51E0F52E12E08F
:100CC000812F0E94320201E0892B09F400E0F50136
:100CD00081915F01081751F00E94E302F7016083E0
:100CE000718382839383F50131970083F6018081BC
:100CF0000817E1F00E94E302F70140805180628012
:100D0000738064197509860997096B3F7105810520
:100D1000910560F0F60100830E94E302F701608311
:100D2000718382839383812F0E947A041F5FFFEF78
:100D3000CF1ADF0A24E0E20EF11C153009F60E94FA
:100D4000E30200914301109144012091450130914B
:100D50004601601B710B820B930B61367A4E810545
:100D6000910508F4C6C00E94E302609343017093AA
:100D70004401809345019093460182E00E947A04E9
:100D800083E00E947A0484E00E947A040E94EF02C9
:100D9000882349F08091EA018B3028F08D3050F0A3
:100DA00085518230C8F1812C912C20ECA22E2FE7A6
:100DB000B22E1EC06091E50170E090E080E00E94DC
:100DC00019092DEC3CEC4CEC5DE30E94CE096B0163
:100DD0007C016091E40170E090E080E00E941909DC
:100DE0009B01AC01C701B6010E9470084B015C0178
:100DF0000E94EF02882309F474C08091EA018C30CC
:100E000009F482C0D8F48B3091F1C12CD12C80EC44
:100E1000E82E8FE7F82E55C06091E4017091E5014E
:100E200076276727762790E080E00E9417092DEC4F
:100E30003CEC4CEC5DE30E94CE09D8CF855182306A
:100E400020F71091E601612F70E0762F6627662764
:100E50007F778091E701682B90E080E00E9417097E
:100E60002DEC3CEC4CEC5DE30E94CE0969C0609136
:100E7000E60170E090E080E00E9417096B017C01C0
:100E80001091E70117FF0AC0AC019B0160E070E020
:100E900080E89FEB0E946F086B017C011F70612F3F
:100EA00070E090E080E00E9419092DEC3CEC4CECE5
:100EB0005DE30E94CE09A70196010E9470086B01B4
:100EC0007C01A5019401C501B4010E943B0A811176
:100ED00008C0A7019601C701B6010E943B0A8823FA
:100EE000C1F184E990E00E94CE0182E191E00E948C
:100EF0001B04209709F4D7CE0E944B01882309F4E4
:100F0000D2CE0E940000CFCE1091E601612F70E09A
:100F100090E080E00E9417096B017C016091E7017D
:100F20006F7070E090E080E00E9419092DEC3CECBD
:100F30004CEC5DE30E94CE09A70196010E94700867
:100F40006B017C0117FFBDCFF7FAF094F7F8F0942E
:100F5000B8CF8EE890E00E94CE0126013701E894D8
:100F600077F82FEF3FEF4FE75FE7C301B2010E9431
:100F70003B0A81113DC02FEF3FEF4FE75FE7C30111
:100F8000B2010E94DC0818169CF58FE191E00E94E6
:100F90001B0488E890E00E94CE01C501B4010E94C4
:100FA000E1086B01770FEE08FF084AE0C701B601C0
:100FB000F7FE0DC06DE287E491E00E948101662793
:100FC0007727CB016C197D098E099F094AE00E94A1
:100FD000280486E890E00E94CE0182E191E00E9420
:100FE0001B0465E070E080E090E00E94B10281CFD8
:100FF0002FEF3FEF4FE75FE4C701B6010E94C90939
:1010000018161CF483E291E0C2CF2FEF3FEF4FE7B9
:101010005FECC701B6010E94DC0887FDF3CF20E03A
:1010200030E0A901C701B6010E94DC0887FF09C0B2
:101030006DE287E491E00E948101F7FAF094F7F8FD
:10104000F0942AE037ED43EA5BE3C701B6010E9462
:1010500070082B013C010E94E8086B017C010E9492
:1010600017099B01AC01C301B2010E946F082B015B
:101070003C014AE0C701B6010E9428046EE287E401
:1010800091E00E94810120E030E040E251E4C301A0
:10109000B2010E94CE092B013C010E94E8086B01BD
:1010A000F12CE12C4AE0C701B6010E942804C701D7
:1010B000B6010E9417099B01AC01C301B2010E9455
:1010C0006F0820E030E040E251E40E94CE090E9427
:1010D000E80890E080E04AE00E9428045ACF505887
:1010E000BB27AA270E9487080C948F090E948109B8
:1010F00038F00E94880920F039F49F3F19F426F453
:101100000C947E090EF4E095E7FB0C947809E92F26
:101110000E94A00958F3BA1762077307840795075E
:1011200020F079F4A6F50C94C2090EF4E0950B2E8C
:10113000BA2FA02D0B01B90190010C01CA01A00129
:101140001124FF27591B99F0593F50F4503E68F184
:101150001A16F040A22F232F342F4427585FF3CFC5
:10116000469537952795A795F0405395C9F77EF496
:101170001F16BA0B620B730B840BBAF09150A1F0DF
:10118000FF0FBB1F661F771F881FC2F70EC0BA0F65
:10119000621F731F841F48F4879577956795B795ED
:1011A000F7959E3F08F0B0CF9395880F08F09927E8
:1011B000EE0F9795879508950E94540908F481E0F1
:1011C00008950E94E8086894B1110C94C309089529
:1011D0000E94A80988F09F5798F0B92F9927B75116
:1011E000B0F0E1F0660F771F881F991F1AF0BA95CB
:1011F000C9F714C0B13091F00E94C209B1E008955E
:101200000C94C209672F782F8827B85F39F0B93F4F
:10121000CCF3869577956795B395D9F73EF490957D
:101220008095709561957F4F8F4F9F4F0895E894FB
:1012300009C097FB3EF490958095709561957F4F1E
:101240008F4F9F4F9923A9F0F92F96E9BB279395CC
:10125000F695879577956795B795F111F8CFFAF4DC
:10126000BB0F11F460FF1BC06F5F7F4F8F4F9F4F0D
:1012700016C0882311F096E911C0772321F09EE86B
:10128000872F762F05C0662371F096E8862F70E0D1
:1012900060E02AF09A95660F771F881FDAF7880FAB
:1012A0009695879597F90895990F0008550FAA0B01
:1012B000E0E8FEEF16161706E807F907C0F0121669
:1012C0001306E407F50798F0621B730B840B950B6C
:1012D00039F40A2661F0232B242B252B21F40895C1
:1012E0000A2609F4A140A6958FEF811D811D08955E
:1012F00097F99F6780E870E060E008959FEF80ECC9
:10130000089500240A94161617061806090608956B
:1013100000240A9412161306140605060895092ED1
:101320000394000C11F4882352F0BB0F40F4BF2B40
:1013300011F460FF04C06F5F7F4F8F4F9F4F089580
:1013400057FD9058440F551F59F05F3F71F0479576
:10135000880F97FB991F61F09F3F79F0879508955B
:10136000121613061406551FF2CF4695F1DF08C07A
:10137000161617061806991FF1CF86957105610597
:1013800008940895E894BB2766277727CB0197F93F
:1013900008950E94540908F48FEF08950E94E1090E
:1013A0000C948F090E94810938F00E94880920F06E
:1013B000952311F00C9478090C947E0911240C9457
:1013C000C3090E94A00970F3959FC1F3950F50E0E7
:1013D000551F629FF001729FBB27F00DB11D639FE7
:1013E000AA27F00DB11DAA1F649F6627B00DA11D8D
:1013F000661F829F2227B00DA11D621F739FB00D33
:10140000A11D621F839FA00D611D221F749F3327A2
:10141000A00D611D231F849F600D211D822F762F3B
:101420006A2F11249F5750409AF0F1F088234AF018
:10143000EE0FFF1FBB1F661F771F881F9150504084
:10144000A9F79E3F510580F00C9478090C94C309CC
:101450005F3FE4F3983ED4F3869577956795B7950B
:10146000F795E7959F5FC1F7FE2B880F911D969525
:10147000879597F908950E945409880B990B089550
:10148000A1E21A2EAA1BBB1BFD010DC0AA1FBB1F88
:10149000EE1FFF1FA217B307E407F50720F0A21BFA
:1014A000B30BE40BF50B661F771F881F991F1A9467
:1014B00069F760957095809590959B01AC01BD0191
:1014C000CF010895EE0FFF1F0590F491E02D0994D0
:1014D000F894FFCF000000008101E1000E01E90156
:1014E0003F011D0131010D0A003D0048004C003054
:0C14F0002E3100696E66006F7666000009
:107E0000112484B714BE81FFF0D085E080938100F7
:107E100082E08093C00088E18093C10086E0809377
:107E2000C20080E18093C4008EE0C9D0259A86E02C
:107E300020E33CEF91E0309385002093840096BBD3
:107E4000B09BFECF1D9AA8958150A9F7CC24DD24C4
:107E500088248394B5E0AB2EA1E19A2EF3E0BF2EE7
:107E6000A2D0813461F49FD0082FAFD0023811F036
:107E7000013811F484E001C083E08DD089C08234E0
:107E800011F484E103C0853419F485E0A6D080C0E4
:107E9000853579F488D0E82EFF2485D0082F10E0AE
:107EA000102F00270E291F29000F111F8ED06801E7
:107EB0006FC0863521F484E090D080E0DECF843638
:107EC00009F040C070D06FD0082F6DD080E0C81688
:107ED00080E7D80618F4F601B7BEE895C0E0D1E017
:107EE00062D089930C17E1F7F0E0CF16F0E7DF06D8
:107EF00018F0F601B7BEE89568D007B600FCFDCFD4
:107F0000A601A0E0B1E02C9130E011968C91119780
:107F100090E0982F8827822B932B1296FA010C0160
:107F200087BEE89511244E5F5F4FF1E0A038BF0790
:107F300051F7F601A7BEE89507B600FCFDCF97BE46
:107F4000E89526C08437B1F42ED02DD0F82E2BD052
:107F50003CD0F601EF2C8F010F5F1F4F84911BD097
:107F6000EA94F801C1F70894C11CD11CFA94CF0C13
:107F7000D11C0EC0853739F428D08EE10CD085E9AC
:107F80000AD08FE07ACF813511F488E018D01DD067
:107F900080E101D065CF982F8091C00085FFFCCF94
:107FA0009093C60008958091C00087FFFCCF809118
:107FB000C00084FD01C0A8958091C6000895E0E648
:107FC000F0E098E1908380830895EDDF803219F02E
:107FD00088E0F5DFFFCF84E1DECF1F93182FE3DFCA
:107FE0001150E9F7F2DF1F91089580E0E8DFEE27F6
:047FF000FF270994CA
:027FFE00040479
:00000001FF
